:020000040000FA
:10000000C9EF24F0120012001AEF00F012000300F2
:10001000F84B0000E00C000018000000F44B00005A
:10002000FC01000004000000144A0000000700006A
:10003000E0010000DACFE4FFE2CFDAFFE9CFE4FF2E
:10004000EACFE4FFF6CFE4FFF7CFE4FFF5CFE4FF1C
:10005000F3CFE4FFF4CFE4FFFACFE4FF00EE00F0CB
:10006000140EE80403E3EECFE4FFFBD700EE14F038
:10007000080EE80403E3EECFE4FFFBD7E652A350FB
:10008000200B3CE0A450200B39E0C1EC23F001012F
:100090008A6F71A405D0719E718E8A6B8F6B906B85
:1000A00071A205D0719871888A6B8F6B906B0D0E61
:1000B0008A5D23E18F51901120E1000E9325E96EB6
:1000C000010E9421EA6EEF6A020E8F6F906BA39A75
:1000D00093C195F194C196F1936B946B7F0E96AF9B
:1000E00002D0D89003D0955D000E965906E3936B2D
:1000F000946B030E8F6F906BA39AA49A9D50200B64
:100100003CE09E50200B39E0E0EC23F00101896FC8
:10011000ABA403D0AB9EAB8E896BABA203D0AB98E4
:10012000AB88896B0D0E895D1AE00A0E895D17E0B8
:10013000800E92AF02D0D89003D0915D000E9259FC
:100140000EE2000E9125E96E0B0E9221EA6E89C136
:10015000EFFF912B000E92238D6B8E6B0DD09D9A2D
:10016000000E9125E96E0B0E9221EA6EEF6A010EE8
:100170008D6F8E6B916B926B9E9AA050020B17E065
:10018000A150020B14E001019707000E985B9751F4
:1001900098110CE1010E8B6F8C6BB190000EE66E26
:1001A000E66AFFEC23F0E552E552A092A192E552F7
:1001B00000EE1BF0080EE80403E3E5CFEDFFFBD7EC
:1001C00000EE13F0140EE80403E3E5CFEDFFFBD7D8
:1001D000E5CFFAFFE5CFF4FFE5CFF3FFE5CFF5FF7D
:1001E000E5CFF7FFE5CFF6FFE5CFEAFFE5CFE9FF83
:1001F000E5CFDAFF1100D9CFE6FFE1CFD9FFFF0E3F
:10020000E76EFD0EDBCF14F0FE0EDBCF15F0E750EE
:100210001416156A1450A96EFD0EDBCF14F0FE0EF5
:10022000DBCF15F015C014F0156A030E1414AA6E76
:10023000A69EA69CA680A85000D0E552E7CFD9FF85
:100240001200D9CFE6FFE1CFD9FF020EE126DE6A28
:10025000DD6AFF0EE76EFD0EDBCF14F0FE0EDBCF86
:1002600015F0E7501416156A1450A96EFD0EDBCF79
:1002700014F0FE0EDBCF15F015C014F0156A030E56
:100280001414AA6EFC0EDB50A86EA69EA684A69C33
:10029000F2AE04D0F29E010EDE6EDD6A550EA76E40
:1002A000AA0EA76EA682A1A8FED7A198A694D9CF20
:1002B000E9FFDACFEAFF010EEE1801E1ED5001E1AE
:1002C000F28E020EE15C02E2E16AE552E16EE55275
:1002D000E7CFD9FF1200D9CFE6FFE1CFD9FFFB0E60
:1002E000DBCFE9FFFC0EDBCFEAFFEF501DE0FB0E9A
:1002F000DBCFE9FFDB2AFC0EDBCFEAFF01E3DB2AE1
:10030000EF50E66EFD0EDBCF14F0DB2AFE0EDBCFE6
:1003100015F001E3DB2A14C0E6FF15C0E6FF91DF0C
:10032000E552E552E552DBD7E552E7CFD9FF12009F
:10033000D9CFE6FFE1CFD9FFE652D950FD0FE96EE4
:10034000FF0EDA20EA6EFF0ED880EE54030EED5455
:1003500001E218D0FD0EDBCFE6FFFE0EDBCFE6FF9D
:100360004ADFE552E552DF6EDF5001E10BD0DFCF0F
:10037000E6FFDCD9E552FD0EDB2AFE0E01E3DB2AA7
:10038000DF50DBE1E80EE66E030EE66EE66AE66A33
:1003900021DAE552E552E552E552E552E552E7CF62
:1003A000D9FF1200D9CFE6FFE1CFD9FF050EE12634
:1003B000F29E000EE66EE66A1EDFE552E552146E0E
:1003C00014C015F0146A14C0DEFF15C0DDFF010E65
:1003D000E66EE66A10DFE552E552E76E000EDFCF0B
:1003E00014F0010EDBCF15F0E7501426000E152295
:1003F000020E14C0DBFF030E15C0DBFF020EDBCFC5
:10040000E6FF030EDBCFE6FF3F0E146E3E0E156EC9
:10041000166A14C0E6FF15C0E6FF16C0E6FFA3C1CA
:10042000E6FFA4C1E6FFBBEC21F0176E070EE15E0C
:100430001750F3CF7CF1F4CF7DF1A3C1E6FFA4C147
:10044000E6FF06D9E552E552F3CF7CF1F4CF7DF11A
:10045000200E146E3E0E156E166A14C0E6FF15C00F
:10046000E6FF16C0E6FFA3C1E6FFA4C1E6FFBBECB2
:1004700021F0176E050EE15E1750F3CF7CF1F4CF3B
:100480007DF1A3C1E6FFA4C1E6FFE2D8E552E55243
:10049000F3CF7CF1F4CF7DF1D950020FE96EDACFC2
:1004A000EAFFFF0ED880EE54030EED5401E235D082
:1004B000020EDE6EDD6ADECF14F0DDCF15F0020E27
:1004C000DBCF16F0030EDBCF17F01650145C17507D
:1004D000155814E2DECFE6FFDDCFE6FF8CDEE552F5
:1004E000E552E76E040EE7CFDBFFDBCFE6FF1ED958
:1004F000E552DF2A010E01E3DB2ADDD757D94C0E86
:100500000B01005D09E1006B0101A76BA86B8D6B0E
:100510008E6B9D8A916B926BF28E050EE15C02E20E
:10052000E16AE552E16EE552E7CFD9FF1200340EE1
:10053000E66EE66A7C0EE66E2CEC23F0E552E552A0
:10054000E55212000F013F9F640EE66EE66A80ECF2
:1005500021F0E552E552340EE66EE66A7C0EE66E58
:10056000F0EC22F0E552E552E5521200D9CFE6FF59
:10057000E1CFD9FF020EE126DE6ADD6AFD0EDBCF98
:10058000F6FFFE0EDBCFF7FF0800F55015E0FD0E7D
:10059000DBCFF6FFFE0EDBCFF7FF0800F550E66E6F
:1005A000C5D8E552DF2A010E01E3DB2AFD0EDB2A66
:1005B000FE0E01E3DB2AE2D7DECF14F0DDCF15F02B
:1005C00014C0F3FF15C0F4FF020EE15C03E200D09B
:1005D000E16AE552E16EE552E7CFD9FF1200D9CFCB
:1005E000E6FFE1CFD9FF020EE126DE6ADD6AFD0EED
:1005F000DBCFF6FFFE0EDBCFF7FF0800F55015E06E
:10060000FD0EDBCFF6FFFE0EDBCFF7FF0800F55047
:10061000E66E9CD8E552DF2A010E01E3DB2AFD0ECF
:10062000DB2AFE0E01E3DB2AE2D7DECF14F0DDCFBA
:1006300015F014C0F3FF15C0F4FF020EE15C03E2F5
:1006400000D0E16AE552E16EE552E7CFD9FF120032
:10065000D9CFE6FFE1CFD9FF020EE126DE6ADD6ADF
:10066000FD0EDBCFE9FFFE0EDBCFEAFFEF5014E01B
:10067000FD0EDBCFE9FFFE0EDBCFEAFFEF50E66EAB
:1006800055D8E552DF2A010E01E3DB2AFD0EDB2AF5
:10069000FE0E01E3DB2AE4D7DECF14F0DDCF15F048
:1006A00014C0F3FF15C0F4FF020EE15C03E200D0BA
:1006B000E16AE552E16EE552E7CFD9FF1200D9CFEA
:1006C000E6FFE1CFD9FF020EE126DE6ADD6AFD0E0C
:1006D000DBCFE9FFFE0EDBCFEAFFEF5014E0FD0EAB
:1006E000DBCFE9FFFE0EDBCFEAFFEF50E66E2ED840
:1006F000E552DF2A010E01E3DB2AFD0EDB2AFE0EA6
:1007000001E3DB2AE4D7DECF14F0DDCF15F014C00F
:10071000F3FF15C0F4FF020EE15C03E200D0E16AD2
:10072000E552E16EE552E7CFD9FF1200D9CFE6FFDF
:10073000E1CFD9FFACA2FED7FE0EDBCFE6FF6AEC1D
:1007400024F0E552E552E7CFD9FF1200D9CFE6FFFA
:10075000E1CFD9FF72A2FED7FE0EDBCFE6FF53EC4E
:1007600024F0E552E552E7CFD9FF1200D9CFE6FFDA
:10077000E1CFD9FFACA2FED7FD0EDBCFE6FF6AECDE
:1007800024F0E552E552E7CFD9FF1200D9CFE6FFBA
:10079000E1CFD9FF72A2FED7FD0EDBCFE6FF53EC0F
:1007A00024F0E552E552E7CFD9FF12001D0EE66EA8
:1007B0003E0EE66EDBDEE552E55212001D0EE66EE1
:1007C0003E0EE66E0CDFE552E552F3CF7CF1F4CF3E
:1007D0007DF11200D9CFE6FFE1CFD9FFD950FB0F51
:1007E000E96EFF0EDA20EA6ED880000EEE54000E9D
:1007F000EE54000EEE54000EEE540CE2D950FB0FF6
:10080000E96EFF0EDA20EA6EEE06000EEE5AEE5AA0
:10081000EE5AE4D7E552E7CFD9FF1200D9CFE6FF71
:10082000E1CFD9FFFE0EDBCFE6FFA9EC24F0E552C5
:10083000FE0EDBCFE6FFA9EC24F0E552FE0EDBCF87
:10084000E6FFA9EC24F0E552FE0EDBCFE6FFA9ECB3
:1008500024F0E552E552E7CFD9FF1200FFD712008E
:10086000C280C186C194FC0EC1140009C16EC08E45
:10087000C08AC088C096C094C082C0900F01428FC9
:100880004289428B428D1200D9CFE6FFE1CFD9FFDA
:10089000020EE126FD0EDBCF14F0FE0EDBCF15F0CD
:1008A000D89014361536D89014361536010E142407
:1008B000C26E010EE66EE5EC24F0E552F29E07EC06
:1008C00025F002EC25F0000901E0FBD7F0EC24F064
:1008D000F3CFDEFFF4CFDDFFF28EDECF14F0DDCFFD
:1008E00015F014C0F3FF15C0F4FF020EE15C03E243
:1008F00000D0E16AE552E16EE552E7CFD9FF120080
:10090000D596D584D582D590D59AD59C000EE66E25
:10091000E66A37EC24F0E552E552F294F29AD59E5D
:100920001200CD8ACD88CD96CD94CD82CD90D08E3B
:10093000DB0EE66E0B0EE66E1BEC24F0E552E55284
:100940009E90A2989F809D901200BA6ABA92BA8037
:10095000BA8CBA9ABA98BA867D0EBB6E9E929D9258
:100960009F821200B19EB19CB18AB188B196B184C8
:10097000B182B190A192A0921200DB0EE66E0B0E36
:10098000E66EFFEC23F0E552E55201018B6B8C6BB8
:10099000B180A192A282A08212000F013F9F8168C4
:1009A000396B8F0E936EF19E6168386B806A388167
:1009B00038833885CF0E926E826A3A6B800E946EC1
:1009C0001200D9CFE6FFE1CFD9FF0E0EE126F90ED6
:1009D000DBCFDEFFDBCFDDFFFB0EDBCF14F0FC0E49
:1009E000DBCF15F0FD0EDBCF16F0FE0EDBCF17F0E0
:1009F000B00E0C6E0F0E0D6EA10E0E6E350E0F6E3C
:100A000014C007F015C008F016C009F017C00AF0AE
:100A100022EC1BF0FB0E07C0DBFFFC0E08C0DBFF67
:100A2000FD0E09C0DBFFFE0E0AC0DBFFF80EDBCFB8
:100A300016F0000EE76E1618E8AE02D0163403D09A
:100A4000E750D880165402E3070E12D0F80EDBCF21
:100A500017F0160EE76E1718E8AE02D0173403D061
:100A6000E750D880175402E2170E02D0F80EDB28A8
:100A7000146E156A14BE1568080E14C0DBFF090E4B
:100A800015C0DBFF020EDB6A030EDB6AFB0EDBCF59
:100A900014F0FC0EDBCF15F0FD0EDBCF16F0FE0ED2
:100AA000DBCF17F00C6A0D6A0E6A0F6A14C007F0EC
:100AB00015C008F016C009F017C00AF0D6EC1CF0FB
:100AC000010A34E1F90EDBCFE9FFDB2AFA0EDBCFB6
:100AD000EAFF01E3DB2A2D0EEF6EFB0EDBCF14F0F5
:100AE000FC0EDBCF15F0FD0EDBCF16F0FE0EDBCFDC
:100AF00017F00C6A0D6A800E0E6EBF0E0F6E14C0DA
:100B000007F015C008F016C009F017C00AF00BEC8A
:100B10001CF0FB0E07C0DBFFFC0E08C0DBFFFD0E68
:100B200009C0DBFFFE0E0AC0DBFF0BD0F90EDBCFE6
:100B3000E9FFDB2AFA0EDBCFEAFF01E3DB2A200E16
:100B4000EF6EFB0EDBCF14F0FC0EDBCF15F0FD0ECD
:100B5000DBCF16F0FE0EDBCF17F00C6A0D6A0E6AC3
:100B60000F6A14C007F015C008F016C009F017C0CE
:100B70000AF0CDEC1CF0010A4AE1FB0EDBCF14F0C9
:100B8000FC0EDBCF15F0FD0EDBCF16F0FE0EDBCF3B
:100B900017F00C6A0D6A800E0E6E3F0E0F6E14C0B9
:100BA00007F015C008F016C009F017C00AF0D6EC1F
:100BB0001CF0010A2CE1146A156A200E166E410E13
:100BC000176ED950FB0FE96EFF0EDA20EA6EEECFFA
:100BD00007F0EECF08F0EECF09F0EFCF0AF014C027
:100BE0000CF015C00DF016C00EF017C00FF00BEC96
:100BF0001CF00AC0EDFF09C0EDFF08C0EDFF07C003
:100C0000EFFF020EDB06030E01E2DB06B6D7FB0E9A
:100C1000DBCF14F0FC0EDBCF15F0FD0EDBCF16F0B2
:100C2000FE0EDBCF17F00C6A0D6A200E0E6E410E21
:100C30000F6E14C007F015C008F016C009F017C0F9
:100C40000AF0D6EC1CF0010A2EE0FB0EDBCF14F00C
:100C5000FC0EDBCF15F0FD0EDBCF16F0FE0EDBCF6A
:100C600017F00C6A0D6A200E0E6E410E0F6E14C046
:100C700007F015C008F016C009F017C00AF0B8EC6C
:100C80001BF0FB0E07C0DBFFFC0E08C0DBFFFD0EF8
:100C900009C0DBFFFE0E0AC0DBFF020EDB2A030EDB
:100CA00001E3DB2AB4D7020EDBCF14F0030EDBCF57
:100CB00015F0D950080FE96EDACFEAFF1450EE268E
:100CC0001550ED22010EF36E040EF3CFDBFF050E7F
:100CD000DB6A040EDBCF08F0050EDBCF09F00EEC6B
:100CE0001BF00A0E07C0DBFF0B0E08C0DBFF0C0E6B
:100CF00009C0DBFF0D0E0AC0DBFF040EDBCF14F0D2
:100D0000050EDBCF15F0080EDBCF16F0090EDBCF9A
:100D100017F015501718E8AE02D0173404D016504B
:100D2000145C175015582EE20A0EDBCF14F00B0E90
:100D3000DBCF15F00C0EDBCF16F00D0EDBCF17F06E
:100D40000C6A0D6A200E0E6E410E0F6E14C007F075
:100D500015C008F016C009F017C00AF0B8EC1BF077
:100D60000A0E07C0DBFF0B0E08C0DBFF0C0E09C02C
:100D7000DBFF0D0E0AC0DBFF040EDB2A050E01E3CC
:100D8000DB2ABBD70A0EDBCF18F00B0EDBCF19F036
:100D90000C0EDBCF1AF00D0EDBCF1BF00C6A0D6AC8
:100DA0000E6A400E0F6E18C007F019C008F01AC086
:100DB00009F01BC00AF0B8EC1BF007C014F008C023
:100DC00015F009C016F00AC017F0D950FB0FE96EF4
:100DD000FF0EDA20EA6EEECF07F0EECF08F0EECF8E
:100DE00009F0EFCF0AF014C00CF015C00DF016C0DA
:100DF0000EF017C00FF022EC1BF00AC0EDFF09C087
:100E0000EDFF08C0EDFF07C0EFFFFB0EDBCF14F0D6
:100E1000FC0EDBCF15F0FD0EDBCF16F0FE0EDBCFA8
:100E200017F00C6A0D6A200E0E6E410E0F6E14C084
:100E300007F015C008F016C009F017C00AF0D6EC8C
:100E40001CF0010A13E0FB0EDB6AFC0EDB6A800E6D
:100E5000F36EFD0EF3CFDBFF3F0EF36EFE0EF3CF0E
:100E6000DBFF020EDB2A030E01E3DB2A020EDBCFDF
:100E700014F0030EDBCF15F00001800E15145FE0B7
:100E8000F90EDBCFE9FFDB2AFA0EDBCFEAFF01E345
:100E9000DB2A300EEF6EF90EDBCFE9FFDB2AFA0E0C
:100EA000DBCFEAFF01E3DB2A2E0EEF6E080EDBCF6D
:100EB00014F0090EDBCF15F0800E151414E0020EAD
:100EC000DBCF16F0030EDBCF17F0080EDB50165CFD
:100ED000146E090EDB501758156E020E14C0DBFF9E
:100EE000030E15C0DBFF040EDB68050EDB68040E85
:100EF000DBCF14F0050EDBCF15F0020EDBCF16F0C2
:100F0000030EDBCF17F017501518E8AE02D01534DA
:100F100004D01450165C1550175811E2F90EDBCFAF
:100F2000E9FFDB2AFA0EDBCFEAFF01E3DB2A300E12
:100F3000EF6E040EDB06050E01E2DB06D8D7040EC9
:100F4000DB6A050EDB6A040EDBCF14F0050EDBCF87
:100F500015F0080EDBCF16F0090EDBCF17F0155099
:100F60001718E8AE02D0173404D01650145C17508E
:100F7000155801E3ACD0FB0EDBCF07F0FC0EDBCF46
:100F800008F0FD0EDBCF09F0FE0EDBCF0AF09EEC81
:100F90001CF0060E08C0DBFF070E09C0DBFF300E99
:100FA000E76E060EDBCF14F0070EDBCF15F0E7502F
:100FB0001426000E1522F90EDBCFE9FFDB2AFA0E0C
:100FC000DBCFEAFF01E3DB2A14C0EFFF040EDBCF27
:100FD00014F0050EDBCF15F0020EDB50141803E100
:100FE000030EDB5015180BE1F90EDBCFE9FFDB2A0E
:100FF000FA0EDBCFEAFF01E3DB2A2E0EEF6E060EC0
:10100000DBCF08F0070EDBCF09F00EEC1BF00A0E69
:1010100007C0DBFF0B0E08C0DBFF0C0E09C0DBFFB7
:101020000D0E0AC0DBFF07C014F008C015F009C0A0
:1010300016F00AC017F0D950FB0FE96EFF0EDA2048
:10104000EA6EEECF07F0EECF08F0EECF09F0EFCF6B
:101050000AF014C00CF015C00DF016C00EF017C049
:101060000FF021EC1BF00AC0EDFF09C0EDFF08C036
:10107000EDFF07C0EFFF146A156A200E166E410ED1
:10108000176ED950FB0FE96EFF0EDA20EA6EEECF35
:1010900007F0EECF08F0EECF09F0EFCF0AF014C062
:1010A0000CF015C00DF016C00EF017C00FF00BECD1
:1010B0001CF00AC0EDFF09C0EDFF08C0EDFF07C03E
:1010C000EFFF040EDB2A050E01E3DB2A3CD7F90E05
:1010D000DBCFE9FFFA0EDBCFEAFFEF6ADECF14F0D9
:1010E000DDCF15F014C0F3FF15C0F4FF0E0EE15C68
:1010F00003E200D0E16AE552E16EE552E7CFD9FFA5
:101100001200D9CFE6FFE1CFD9FF020EE126FE0E95
:10111000DB50F00BDF6EDF380F0BDF6E300EDF249D
:10112000DF6EDF50390803E2070EDF24DF6EFE0EAC
:10113000DB500F0B300FE76E010EE7CFDBFFDB500C
:10114000390807E2010EDB50070FE76E010EE7CF0B
:10115000DBFFDFCFE6FF96EC03F0E552010EDBCFBD
:10116000E6FF96EC03F0E552020EE15C02E2E16A72
:10117000E552E16EE552E7CFD9FF120086C1E6FFE6
:101180008FEC18F0E5520B010D6BE66A000EE66E6F
:101190000B0EE66EE3EC1AF0E552E552E552000E56
:1011A000E66E0B0EE66E5FEC03F0E552E552F3CF10
:1011B0007CF1F4CF7DF1DEEC03F0050EE66E2A0E35
:1011C000E66E79EC18F0E552E552300E0101156A31
:1011D0009B25146E9C51152214C0E6FF15C0E6FF36
:1011E000B6EC16F0E552E5521200010E0101866FD1
:1011F000876B050EE66EE66A79EC18F0E552E5526B
:101200000E0EE66E3E0EE66E04EC17F0E552E55269
:10121000A00EE66E860EE66E010EE66EE66AEAEC5B
:1012200003F0E552E552E552E552DEEC03F0010130
:101230009B6B9C6B100E976F986BBDEC04F00101DB
:10124000896B8D6B8E6B9E9A916B926B786B796BC1
:101250000D0E785D000E79590BE2000E7825E96ECF
:101260000B0E7921EA6EEF6A782B000E7923F0D706
:101270000B0EE66E3E0EE66EB6EC02F0E552E5525F
:10128000F3CFC3F1F4CFC4F1AAEC21F001018951ED
:1012900003E18B518C11FAE0020EE66EE66A080E4D
:1012A000146E3E0E156E166A14C0E6FF15C0E6FFFA
:1012B00016C0E6FF000EE66E0B0EE66EF1EC20F0B7
:1012C000176E070EE15E1750000904E101019B2B28
:1012D000000E9C23FF0EE66E3D0EE66EEFEC02F074
:1012E000E552E552F3CFC3F1F4CFC4F147DF01017A
:1012F000010E9B1901E19C5103E0F36AF46A44D1A9
:10130000020E866F876B100E976F986BBDEC04F022
:101310000101896B8D6B8E6B9E9A916B926B786BD2
:10132000796B0D0E785D000E79590BE2000E782571
:10133000E96E0B0E7921EA6EEF6A782B000E7923A5
:10134000F0D70B01006BF40EE66E3D0EE66EB6ECC8
:1013500002F0E552E552F3CFC3F1F4CFC4F1AAECA9
:1013600021F00101895103E18B518C11FAE0080E43
:10137000E66EE66AEB0E146E3D0E156E166A14C02C
:10138000E6FF15C0E6FF16C0E6FF000EE66E0B0E88
:10139000E66EF1EC20F0176E070EE15E17500009C3
:1013A00004E101019B2B000E9C23E20EE66E3D0E34
:1013B000E66EEFEC02F0E552E552F3CFC3F1F4CF65
:1013C000C4F1DCDE0101020E9B1901E19C5103E036
:1013D000F36AF46AD9D0030E866F876B100E976F8D
:1013E000986BBDEC04F00101896B8D6B8E6B9E9A3E
:1013F000916B926B786B796B0D0E785D000E79595D
:101400000BE2000E7825E96E0B0E7921EA6EEF6A89
:10141000782B000E7923F0D7CF0EE66E3D0EE66EE8
:10142000B6EC02F0E552E552F3CFC3F1F4CFC4F1CC
:10143000AAEC21F00101895103E18B518C11FAE0F2
:10144000090EE66EE66AC50E146E3D0E156E166A3E
:1014500014C0E6FF15C0E6FF16C0E6FF000EE66EFC
:101460000B0EE66EF1EC20F0176E070EE15E1750E2
:10147000000904E101019B2B000E9C23BC0EE66ECB
:101480003D0EE66EEFEC02F0E552E552F3CFC3F10C
:10149000F4CFC4F173DE0101030E9B1901E19C51ED
:1014A00003E0F36AF46A70D0040E866F876B100E47
:1014B000976F986BBDEC04F00101896B8D6B8E6B9F
:1014C0009E9A916B926B786B796B0D0E785D000E26
:1014D00079590BE2000E7825E96E0B0E7921EA6E40
:1014E000EF6A782B000E7923F0D70B01006BB10E59
:1014F000E66E3D0EE66EB6EC02F0E552E552F3CF35
:10150000C3F1F4CFC4F1AAEC21F00101895103E148
:101510008B518C11FAE0090EE66EE66AA70E146E86
:101520003D0E156E166A14C0E6FF15C0E6FF16C024
:10153000E6FF000EE66E0B0EE66EF1EC20F0176E85
:10154000070EE15E1750000904E101019B2B000E1C
:101550009C239E0EE66E3D0EE66EEFEC02F0E55229
:10156000E552F3CFC3F1F4CFC4F108DE0101040E5C
:101570009B1901E19C5103E0F36AF46A05D09BC119
:10158000F3FF9CC1F4FF00D012000101896B916B45
:10159000926B786B796B0D0E785D000E79590BE2CA
:1015A000000E7825E96E0B0E7921EA6EEF6A782B32
:1015B000000E7923F0D79E9A9D8A86C1E6FFE66ADF
:1015C00079EC18F0E552E5528F0EE66E3D0EE66EB0
:1015D00004EC17F0E552E55286C1E6FFE66A79ECC5
:1015E00018F0E552E552200EE66E030EE66E80EC32
:1015F00021F0E552E5520101923504E291510008D3
:10160000000E925520E20B010D6B000EE66E0B0EE4
:10161000E66E5FEC03F0E552E552F3CF7CF1F4CFD8
:101620007DF1DEEC03F00101916B926B9E9A9D9A25
:10163000E66A000EE66E0B0EE66EE3EC1AF0E5527B
:10164000E552E55208D0800EE66E3D0EE66E04ECE3
:1016500017F0E552E5521200DEEC03F0010E010135
:10166000866F876B0B0E146E3E0E156E166A14C0D5
:10167000E6FF15C0E6FF16C0E6FFFE0EE66EE66862
:1016800060EC22F0176E050EE15E1750F3CF7CF18F
:10169000F4CF7DF17ADF020E0101866F876BF40EC5
:1016A000146E3D0E156E166A14C0E6FF15C0E6FFF7
:1016B00016C0E6FFFE0EE66EE66860EC22F0176EDE
:1016C000050EE15E1750F3CF7CF1F4CF7DF15DDFC5
:1016D000030E0101866F876BCF0E146E3D0E156EE3
:1016E000166A14C0E6FF15C0E6FF16C0E6FFFE0E40
:1016F000E66EE66860EC22F0176E050EE15E1750AC
:10170000F3CF7CF1F4CF7DF140DF040E0101866F51
:10171000876BB10E146E3D0E156E166A14C0E6FF8F
:1017200015C0E6FF16C0E6FFFE0EE66EE66860EC4A
:1017300022F0176E050EE15E1750F3CF7CF1F4CF67
:101740007DF123DF050E0101866F876B12009D9AE4
:10175000E0EC23F00101896F896B916B926B956BC3
:10176000966B0B01006B0501000E536F0B0E546F4F
:101770009E9A01018D6B8E6B9D8A9E9A1200700E4F
:10178000D36E9B6A9B9C0101916B926B936B946BE4
:10179000D48DD4898D6B8E6B8F6B906B896B8A6BBC
:1017A0000C01F66BF76B0101800EA36F0B0EA46F9B
:1017B000CDEC04F0F40EE66E010EE66E80EC21F046
:1017C000E552E5520101786B796B740E785D000E7D
:1017D000795912E2000E7825E96E0C0E7921EA6E35
:1017E000EF6A000E7825E96E010E7921EA6EEF6A44
:1017F000782B000E7923E9D7AADF97EC02F0A2EC50
:1018000002F00C0EE66EE66AC6EC03F0E552E55215
:10181000DC0EE66E050EE66E80EC21F0E552E55238
:10182000DEEC03F0A58A7198A39A0101800EA36FE4
:101830000B0EA46FF2CC14F0F3CC15F0166A14C0A2
:10184000E6FF15C0E6FF16C0E6FFA3C1E6FFA4C190
:10185000E6FF10EC21F0176E050EE15E1750A3C1F4
:10186000E6FFA4C1E6FF5FEC03F0E552E552F3CFDB
:101870007CF1F4CF7DF10101800EA36F0B0EA46FFC
:10188000F4CC14F0F5CC15F0166A14C0E6FF15C0C0
:10189000E6FF16C0E6FFA3C1E6FFA4C1E6FF10EC19
:1018A00021F0176E050EE15E1750A3C1E6FFA4C13B
:1018B000E6FF5FEC03F0E552E552F3CF7CF1F4CFA5
:1018C0007DF10101800EA36F0B0EA46FE8CC14F024
:1018D000E9CC15F0166A14C0E6FF15C0E6FF16C085
:1018E000E6FFA3C1E6FFA4C1E6FF10EC21F0176EEE
:1018F000050EE15E1750A3C1E6FFA4C1E6FF5FEC51
:1019000003F0E552E552F3CF7CF1F4CF7DF1010114
:10191000800EA36F0B0EA46FE0CC14F0E1CC15F099
:10192000166A14C0E6FF15C0E6FF16C0E6FFA3C1A5
:10193000E6FFA4C1E6FF10EC21F0176E050EE15E94
:101940001750A3C1E6FFA4C1E6FF5FEC03F0E55228
:10195000E552F3CF7CF1F4CF7DF171EC17F0640E1A
:10196000E66EE66A80EC21F0E552E552E66A8FEC1D
:1019700018F0E552710EE66E3D0EE66E04EC17F0BF
:10198000E552E552010EE66E8FEC18F0E552620E5C
:10199000E66E3D0EE66E04EC17F0E552E552640E7D
:1019A000E66EE66A80EC21F0E552E552020EE66E44
:1019B0008FEC18F0E552530EE66E3D0EE66E04EC29
:1019C00017F0E552E552640EE66EE66A80EC21F00F
:1019D000E552E552030EE66E8FEC18F0E552440E28
:1019E000E66E3D0EE66E04EC17F0E552E552640E2D
:1019F000E66EE66A80EC21F0E552E552040EE66EF2
:101A00008FEC18F0E552350EE66E3D0EE66E04ECF6
:101A100017F0E552E552640EE66EE66A80EC21F0BE
:101A2000E552E552050EE66E8FEC18F0E552260EF3
:101A3000E66E3D0EE66E04EC17F0E552E552640EDC
:101A4000E66EE66A80EC21F0E552E552D00EE66ED5
:101A5000070EE66E80EC21F0E552E552A4AA05D00F
:101A6000C1EC23F001018A6FF9D701018A6B8F6BFA
:101A7000906B006B956B966BDEEC03F00101800EB2
:101A8000A36F0B0EA46F130E146E3D0E156E166A27
:101A900014C0E6FF15C0E6FF16C0E6FFA3C1E6FFCF
:101AA000A4C1E6FF10EC21F0176E050EE15E1750A1
:101AB000A3C1E6FFA4C1E6FF5FEC03F0E552E552E7
:101AC000AAEC21F0AAEC21F0AAEC21F0AB889E9AB6
:101AD0009D8A9F8AD08EF28CF28E9EAA05D0E0EC71
:101AE00023F00101896FF9D7E80EE66E030EE66E6A
:101AF00080EC21F0E552E552AAEC21F0B2EC04F0C2
:101B00000101800EA36F0B0EA46FE20E146E3C0E4B
:101B1000156E166A14C0E6FF15C0E6FF16C0E6FF94
:101B2000A3C1E6FFA4C1E6FF10EC21F0176E050E7D
:101B3000E15E1750A3C1E6FFA4C1E6FF5FEC03F02E
:101B4000E552E552AAEC21F0F5EC08F0F3CF80F174
:101B5000F4CF81F1AAEC21F0E66AE66A79EC18F09C
:101B6000E552E5520101040E801901E181512FE196
:101B7000D30EE66E3C0EE66E04EC17F0E552E5522D
:101B80000101800EA36F0B0EA46F80C1E6FF81C11F
:101B9000E6FFA50E146E3C0E156E166A14C0E6FF25
:101BA00015C0E6FF16C0E6FFA3C1E6FFA4C1E6FF2D
:101BB000BBEC21F0176E070EE15E1750A3C1E6FFE4
:101BC000A4C1E6FF5FEC03F0E552E5522ED0960E7D
:101BD000E66E3C0EE66E04EC17F0E552E5520101AC
:101BE000800EA36F0B0EA46F80C1E6FF81C1E6FFDC
:101BF000670E146E3C0E156E166A14C0E6FF15C013
:101C0000E6FF16C0E6FFA3C1E6FFA4C1E6FFBBECFA
:101C100021F0176E070EE15E1750A3C1E6FFA4C1C5
:101C2000E6FF5FEC03F0E552E552050EE66E8FEC41
:101C300018F0E552040EE66E8FEC18F0E552030E34
:101C4000E66E8FEC18F0E552020EE66E8FEC18F09F
:101C5000E552010EE66E8FEC18F0E552580EE66E76
:101C60003C0EE66E04EC17F0E552E5520101800EE1
:101C7000A36F0B0EA46F2E0E146E3C0E156E166A1B
:101C800014C0E6FF15C0E6FF16C0E6FFA3C1E6FFDD
:101C9000A4C1E6FFBBEC21F0176E050EE15E175004
:101CA000A3C1E6FFA4C1E6FF5FEC03F0E552E552F5
:101CB00030EC04F0AAEC21F0000EE66EE66A44EC8B
:101CC00004F0E552E552F3CFCBF1F4CFCCF10101B2
:101CD000400ED880CB55030ECC5504E2400ECB6F9E
:101CE000030ECC6F200ECB5D020ECC5904E2200E09
:101CF000CB6F020ECC6FCBC108F0CCC109F00CEC5D
:101D00001BF007C018F008C019F009C01AF00AC08B
:101D10001BF0CD0E0C6ECC0E0D6E0E6E3E0E0F6EC9
:101D200018C007F019C008F01AC009F01BC00AF06B
:101D30000BEC1CF007C014F008C015F009C016F039
:101D40000AC017F00C6A800E0D6E880E0E6E430EE0
:101D50000F6E14C007F015C008F016C009F017C0C8
:101D60000AF021EC1BF007C0D5F108C0D6F109C07C
:101D7000D7F10AC0D8F1D5C1E1F1D6C1E2F1D7C19E
:101D8000E3F1D8C1E4F1100EE66E270EE66EE66AC6
:101D9000E66AEAEC03F0E552E552E552E552010E3F
:101DA000E66EE66A44EC04F0E552E552F3CFCDF17D
:101DB000F4CFCEF10101960ED880CD55000ECE5550
:101DC00003E2960ECD6FCE6BCDC108F0CEC109F007
:101DD0000CEC1BF007C014F008C015F009C016F099
:101DE0000AC017F0CD0E0C6ECC0E0D6E0E6E3E0EB0
:101DF0000F6E14C007F015C008F016C009F017C028
:101E00000AF00BEC1CF007C0D9F108C0DAF109C0E8
:101E1000DBF10AC0DCF1D9C1E5F1DAC1E6F1DBC1E1
:101E2000E7F1DCC1E8F10101800EA36F0B0EA46F96
:101E3000CDC1E6FFCEC1E6FFCBC1E6FFCCC1E6FFD8
:101E4000050E146E3C0E156E166A14C0E6FF15C022
:101E5000E6FF16C0E6FFA3C1E6FFA4C1E6FFBBECA8
:101E600021F0176E090EE15E1750A3C1E6FFA4C171
:101E7000E6FF5FEC03F0E552E5520101800EA36F2F
:101E80000B0EA46FEC0E146E3B0E156E166A14C08A
:101E9000E6FF15C0E6FF16C0E6FFA3C1E6FFA4C13A
:101EA000E6FF10EC21F0176E050EE15E1750A3C19E
:101EB000E6FFA4C1E6FF5FEC03F0E552E552010145
:101EC000800EA36F0B0EA46FAAEC21F040DC71888A
:101ED000A38A01017E6B7F6B0101010E8D1901E167
:101EE0008E510CE1000EE66E0B0EE66E5FEC03F019
:101EF000E552E552DEEC03F02ADCEED77E2B000E35
:101F00007F2381B2B8D0240EE66E96EC03F0E55242
:101F1000240EE66E96EC03F0E552240EE66E96EC87
:101F200003F0E5520D0EE66E96EC03F0E5520A0E54
:101F3000E66EE66A80EC21F0E552E5520101800E82
:101F4000A36F0B0EA46FE90E146E3B0E156E166A8E
:101F500014C0E6FF15C0E6FF16C0E6FFA3C1E6FF0A
:101F6000A4C1E6FF10EC21F0176E050EE15E1750DC
:101F7000A3C1E6FFA4C1E6FF28EC03F0E552E55259
:101F80000D0EE66E96EC03F0E5520A0EE66EE66A7A
:101F900080EC21F0E552E5520101010E8D1901E1BD
:101FA0008E514CE1800EA36F0B0EA46F310E0B010E
:101FB000005D16E1DC0E146E3B0E156E166A14C041
:101FC000E6FF15C0E6FF16C0E6FFA3C1E6FFA4C109
:101FD000E6FF10EC21F0176E050EE15E175015D0EC
:101FE000CE0E146E3B0E156E166A14C0E6FF15C0B9
:101FF000E6FF16C0E6FFA3C1E6FFA4C1E6FF10ECB2
:1020000021F0176E050EE15E1750DEEC03F0000EB6
:10201000E66E0B0EE66E5FEC03F0E552E552A3C1EF
:10202000E6FFA4C1E6FF5FEC03F0E552E5520D0EBA
:10203000E66EA6EC03F0E552DEEC03F02D0EE66E44
:1020400096EC03F0E5522D0EE66E96EC03F0E552A9
:102050002D0EE66E96EC03F0E5520D0EE66E96EC54
:1020600003F0E5520A0EE66EE66A80EC21F0E552D6
:10207000E552A7EC0BF00101010E8F1901E190511F
:102080005AE1000EE66E010EE66E5FEC03F0E552DB
:10209000E5520D0EE66EA6EC03F0E552520E01017C
:1020A000005D0FE1410E016F01510BE05A0E025D20
:1020B00008E1000EE66E010EE66E28EC03F0E55234
:1020C000E552550E0101005D0CE1230E126F125115
:1020D00008E0000EE66E010EE66E28EC03F0E55215
:1020E000E552520E0101005D0FE1440E016F0151F6
:1020F0000BE0310E035D08E1000EE66E010EE66EA8
:1021000028EC03F0E552E552520E0101005D0FE1AB
:10211000440E016F01510BE0300E035D08E1000E2B
:10212000E66E010EE66E28EC03F0E552E552010181
:10213000006B8F6B906B2C0EE66E010EE66E80ECE2
:1021400021F0E552E552C8D61200E1EC15F0FB0E85
:10215000DBCFF3FFDB06F35000090AE02FEC16F0AB
:10216000FA0E9AEC16F0F3E1151CF1E1010E01D024
:10217000000E10EF16F0E1EC15F03B0EE12402E347
:10218000E168E652E16E010EDB6A020EDB6AF90ECF
:10219000DBCFF6FFFA0EDBCFF7FFFB0EDBCFF8FF4E
:1021A0000800F550DF6EDF5002E134EF15F0250E28
:1021B000DF5C02E027EF15F0030EDB6A040EDB6A3A
:1021C000050EDB6A060EDB6A070EDB6A49EC15F0CA
:1021D0002D0EDF5C0CE02B0EDF5C09E0200EDF5CD7
:1021E00006E0230EDF5C03E0300EDF5C1AE1DF5017
:1021F000300A14E0130A0FE0030A0AE00B0A05E0B4
:10220000060AE4E1030EDB80E1D7030EDB82DED7B2
:10221000030EDB84DBD7030EDB86D8D7030EDB8807
:10222000D5D72A0EDF5C1BE145EC15F093EC15F0D9
:1022300010E0030EDB8008680968130EDBCF0DF099
:10224000140EDBCF0EF0BAEC1DF0040E06C0DBFF5F
:1022500003D0130E7CEC15F049EC15F00BD0090EF1
:10226000DB6AEAEC15F003E05EEC16F0FAD7090E33
:102270007CEC15F0030EDBB0DB982E0EDF5C1BE16F
:1022800049EC15F02A0EDF5C0BE145EC15F093EC00
:1022900015F003E1130ECEEC15F049EC15F00BD060
:1022A000090EDB6AEAEC15F003E05EEC16F0FAD7F3
:1022B000090ECEEC15F0680EDF5C07E149EC15F075
:1022C000680EDF5C1DE1030E18D0740EDF5C17E0B2
:1022D0007A0EDF5C14E0480EDF5C06E0540EDF5C33
:1022E00003E05A0EDF5C02E1020E07D06C0EDF5CE9
:1022F00003E06A0EDF5C04E1010E21EC16F0C9DB9D
:10230000DF506E0A01E17FD31E0A01E192D1200A5B
:1023100001E18FD13F0A01E149D11A0A01E146D119
:102320000D0A01E143D1200A01E140D13A0A01E15D
:102330003DD1200A01E13AD1260A01E135D10D0A49
:1023400001E132D11A0A01E1D9D0200A4AE0300A6B
:102350001FE0460A0EE0250A01E083D3D950F90FA9
:10236000E96EFF0EDA20EA6E010EEE5E000EEE5A06
:10237000EE5A2FEC16F0250EE66E95DB03E1151CE8
:1023800001E169D32BEC16F001E26BD3DB2A69D3B0
:10239000080EDB6A040EDB50010806E2040EDB04C3
:1023A000F3EC15F0DB508BDB080EDB5009E0030E7D
:1023B000DB50010B05E172DB01E04DD3080EDB6A57
:1023C00064DBEFCFDFFFA3EC16F003E1151C01E1A6
:1023D00042D32BEC16F001E3DB2A60DB01E141D3B1
:1023E0003AD3070EDB5002080FE16FEC16F0030E34
:1023F00036EC16F00E0EEECFDBFF0F0EEECFDBFF4E
:10240000100EEECFDBFF20D0F70EDBCF17F0F80E6B
:10241000DBCF18F0020E175E000E185AF70E17C029
:10242000DBFFF80E18C0DBFF17C0E9FF18C0EAFF9A
:1024300026EC16F0166A0E0E14C0DBFF0F0E15C048
:10244000DBFF100E16C0DBFF0E0EDBCFE6FF0F0E1C
:10245000DBCFE6FF100EDBCFE6FF37EC21F0E552D5
:10246000E552E552130E07C0DBFF140E08C0DBFF78
:10247000060EDB5005E0130E6AEC16F001E26ADB93
:102480008EEC16F002E2130E37DB51EC16F006E08C
:10249000040E6AEC16F002E2050E2EDB030EDBB032
:1024A00005D0FCDA01E0D7D2080EDB6A090EDB6A40
:1024B0000E0EDBCFF6FF0F0EDBCFF7FF100EDBCFDC
:1024C000F8FF0800F550DF6EDF5014E094EC16F0D2
:1024D00011E2A3EC16F003E1151C01E1BCD2BBDB59
:1024E00001E3DB2A090EDB2AD9500E0FE96E000E3C
:1024F000CBDBE7D7D3DA01E1B4D2ADD2C6DA110E25
:10250000EECFDBFF120EEDCFDBFF110EDBCFE6FFD0
:10251000120EDBCFE6FF29EC21F0E552E552130E57
:10252000F3CFDBFF140EF4CFDBFF060EDB5004E02D
:10253000130ED0DB01E20EDB8EEC16F002E2130E7E
:10254000DBDAAFDB05E0040EC5DB02E2050ED4DA10
:10255000030EDBB005D0A2DA01E07DD2080EDB6A03
:10256000090EDB6A110EDBCFE9FF120EDBCFEAFFAB
:10257000EFCFDFFFDF5014E0D7DB12E2E4DB03E153
:10258000151C01E168D267DB01E3DB2A090EDB2AB7
:10259000110EDB2ADBCFE9FF120EE8E3DB2AE6D7D8
:1025A0007DDA01E15ED257D2030EDB8E070EDB042B
:1025B00010E195DB040E5ADB0A0EEECFDBFF0B0EAB
:1025C000EECFDBFF0C0EEECFDBFF0D0EEECFDBFF11
:1025D0006CD0070EDB5003082CE1030EDBAE0DD0F0
:1025E000B2DA020E76DAEFCF14F0156A166A176ABD
:1025F00014AE39D01568166835D0F70EDBCF15F05C
:10260000F80EDBCF16F0020E155E000E165AF70E0E
:1026100015C0DBFFF80E16C0DBFF15C0E9FF16C0C2
:10262000EAFFEFCF14F00A0E14C0DBFF0B0EDB6ADB
:1026300038D0070EDB50020809E1030EDBAE04D0F0
:1026400059DB16AE10D00ED055DB0DD0030EDBAE2D
:1026500012D079DA020E3DDAF9DA166A176A15AE87
:1026600002D016681768E2DA0C0E16C0DBFF0D0EFA
:1026700017C0DBFF1AD0F70EDBCF16F0F80EDBCF5A
:1026800017F0020E165E000E175AF70E16C0DBFF8B
:10269000F80E17C0DBFF16C0E9FF17C0EAFFD6DA55
:1026A000C5DA0C0EDB6A0D0EDB6A060EDB5005E1A7
:1026B000010EF36E050EF3CFDBFF150EDB6A160E6F
:1026C000DB6AD950370F146E000EDA20156E390E02
:1026D00014C0DBFF3A0E15C0DBFF380EDB6A080EB4
:1026E000DB6A0A0EAEDADF50780A12E0200A10E048
:1026F000280A0CE0200A0AE03F0A06E00D0A02E080
:10270000200A08E1020E05D0080E03D0080EDF26CD
:10271000100E97DA030EDBBE02D0DB92DB94DB50A7
:10272000800B24E08ADAD890030EEB50000A08E60A
:10273000000EEE5C000EEE58000EEE58000EEE5845
:1027400015E213DA0B680C680D680E6865EC23F06F
:102750000A0E02C0DBFF0B0E03C0DBFF0C0E04C031
:10276000DBFF0D0E05C0DBFF2D0E08D0030EDBA234
:1027700002D02B0E03D0DBA408D0200EF36E170E70
:10278000F3CFDBFF150EDB2A02D0170EDB6A050E36
:10279000DB5003E1B7D901E189D0F20E146E490E86
:1027A000156E000E166E070EDBCF17F0186A196A49
:1027B0001A6A17C00BF018C00CF019C00DF01AC03F
:1027C0000EF0D3D99DEC23F014500224F36E155073
:1027D0000320F46E16500420F86EF4CFF7FFF3CF09
:1027E000F6FF0800090EF5CFDBFF580EDF5C0FE1A6
:1027F000610EF36E090E7BD90AE3200E146E090EEA
:10280000DBCFE7FF1450E75E090EE7CFDBFF070ED3
:10281000DBCF14F0156A166A176A0FDA14C00BF0D2
:1028200015C00CF016C00DF017C00EF0EECF06F07C
:10283000EECF07F0EECF08F0EFCF09F09DEC23F0DC
:1028400009C0EDFF08C0EDFF07C0EDFF06C0EFFFB8
:10285000390EDBCFE9FFDB063A0EDBCFEAFF01E200
:10286000DB06090EDBCFEFFF150EDB2A4BD995E116
:10287000030EDBA61DD06F0EDF5C06E1C1D918E3A5
:10288000150EDB285BDA14D0780EDF5C09E0580EF9
:10289000DF5C06E0620EDF5C03E0420EDF5C08E115
:1028A000020EF36E160EF3CFDBFF02D0150EDB6ABD
:1028B000030EDB50100B0EE0040EDBCF14F0050E00
:1028C000DB50D880145406E2060EDB5003E1040E00
:1028D000DB5034DA95D90AE2050EDBCFE7FF150E9F
:1028E000DB50E75E050EE7CFDBFF02D0050EDB6AAB
:1028F000040EDBCF14F0160E45D9D880145414E220
:10290000160EDBCFE6FF150EDBCFE6FF040EDBCFA6
:10291000E6FF050EDB50E552E75CE552D880E75450
:10292000E552D880E7545FD9030EDB50010B0BE171
:10293000080EDB5008E0B2D801E08DD0080EDB5065
:10294000BED8080EDB6A170EDB5007E088D9170ED9
:10295000F1D903E1151C01E17ED0160EDB5016E023
:102960007ED9300EE66E9FD802E1151C74E077D94F
:10297000DFCFE6FFAEEC22F0E552E552E552F4CFB0
:1029800015F00001F31C02E1151C65E0050EDBCF1C
:1029900014F0160EDB50D880145409E2050EDBCF7C
:1029A000E7FF160EDB50E75E050EE7CFDBFF300ECC
:1029B000E66E050ECBD94FE1390EDB2ADBCFE9FFFE
:1029C0003A0E01E3DB2ADBCFEAFF090EEFCFDBFF94
:1029D000DB500EE044D9090EADD902E1151C3BE0F5
:1029E000390EDB2ADBCFE9FF3A0EEDE3DB2AEBD72A
:1029F00055D831E1160EDBCFE6FF080EC3D8E552FD
:102A0000E7245DD82ED0070EDB50030A1CE0010A34
:102A100014E0030A07E07BD9DBCFEEFF020EDBCF29
:102A2000EDFF1FD0F5D8196A17AE02D018681968E3
:102A30002CD8BCD819C0EEFF14D0EAD817BE18683D
:102A400024D8B4D80ED063D9DBCFEFFF0AD07BD91E
:102A500005E1151C03E1F368F46810D0FCD801E32C
:102A6000DB2A79D9D0EF10F0010EDBCF14F0020E83
:102A7000DBCF15F014C0F3FF15C0F4FF3B0EE15C93
:102A800002E2E16AE552E16ECBD029D9020E36EFBF
:102A900016F061D90800F550DF6E1200200EE66EC8
:102AA000080EA6EF16F0AEEC22F0E552E552E55224
:102AB000F3CF14F0F4CF15F00001F31C1200146EE4
:102AC000156AD950010F4DD91450EE261550ED223C
:102AD0001200185E000E195AF70E18C0DBFFF80E30
:102AE00019C0DBFF18C0E9FF19C0EAFF1200DBCFF5
:102AF000F4FFF350F45C1200DB50E76E040EE7CFF6
:102B0000DBFF12000A0EDBCF14F00B0EDBCF15F04B
:102B10000C0EDBCF16F00D0EDBCF17F01450151096
:102B2000161017101200130EEECFDBFF140EEDCFB0
:102B3000DBFF130EDBCF14F0140EDBCF15F000011A
:102B4000800E15141200F70EDBCF18F0F80EDBCF55
:102B500019F01200050EDB50E66ED950130F01D9A3
:102B6000E552E750EE6EED6A12000A0EDBCF06F07A
:102B70000B0EDBCF07F00C0EDBCF08F00D0EDBCF1A
:102B800009F01200DBCFE6FF150EDBCFE6FF050EE6
:102B9000DB50E552E724E552E7241200DB50CED8A3
:102BA000010EF36E060EF3CFDBFF1200EE50EFCFF7
:102BB000EAFFE96E16C0EEFF17C0EEFF18C0EEFF89
:102BC0001200D9CFE6FFDACFE6FFE1CFD9FFE2CF9F
:102BD000DAFF1200DFCFE6FFE66A97EC24F0E55259
:102BE000E552F3501200E76E080EE7CFDBFF12004C
:102BF000EECF14F0EECF15F0EFCF16F0176A1200FB
:102C0000050EDBCF14F0150EDB50D88014541200E3
:102C1000010EDBCF16F0020EDBCF17F0186A1200A0
:102C2000E552E5CFDAFFE7CFD9FF12000A0E14C054
:102C3000DBFF0B0E15C0DBFF1200D9500A0FB1EFFE
:102C400016F0F36E070EF3CFDBFF1200EECF14F099
:102C5000EFCF15F01200010EDB2A020E1200FC0E5F
:102C6000DBCFE6FFFD0EDBCFE6FF1200145E000EA9
:102C7000155AF70E14C0DBFFF80E15C0DBFF14C0A9
:102C8000E9FF15C0EAFF1200DA20EA6EEF2AEECF64
:102C9000F6FF000EEF22EECFF7FFEF22EECFF8FFA8
:102CA0001200040EDBCFE6FF130EDB50E552E75CAB
:102CB0009ADFDB5004DF060EDB501200090EDB50FA
:102CC0000A0DF350DF24D00FE76E090EE7CFDBFFCC
:102CD00049EF15F0DB50F36E050E77EF15F0F70EA8
:102CE000DBCF14F0F80EDBCF15F01200DFCFE6FFDC
:102CF00053EF15F028DF030EECDEF8EF15F0A5EC2E
:102D000010F0E552E552E552E55200091200BDDE31
:102D1000EE50EFCFEAFFE96E010E1200130EDB500A
:102D2000F36E040E77EF15F0040EDB50F36E090E10
:102D300077EF15F0DBCFE6FF53EF15F0E76E050EEA
:102D4000E7CFDBFF12008BDF76EF16F0DBCFE6FF7D
:102D500086DF7FEF16F0D950F90FE96EFF0E44EFD2
:102D600016F0E96E000EDA20EA6E1200D9CFE6FF07
:102D7000E1CFD9FFFD0EDB500C01C26FC36B200EFB
:102D8000C25D000EC35901E23BD07F0ED880C25510
:102D9000000EC35501E234D0C46BC56B050EC45D93
:102DA000000EC5592AE2C2CCC6FCC3CCC7FC200E1B
:102DB000C65F000EC75B050EC703F3CFC7FCC60393
:102DC000F3CFC6FCF450C727C651C425F66EC751D1
:102DD000C521F76E5D0EF6263E0EF7220800F5CFF0
:102DE000C8FCC96BC8BFC969C8CCE6FF3CD9E5526D
:102DF0000C01C42B000EC523D1D7E66A34D9E552A5
:102E0000E552E7CFD9FF1200D9CFE6FFE1CFD9FFD6
:102E1000020EE126DE6ADD6AFD0EDBCFF6FFFE0E56
:102E2000DBCFF7FF0800F5502EE0FD0EDBCFF6FFFD
:102E3000FE0EDBCFF7FF0800F550E66EE66A96DF80
:102E4000E552E5520000000000000000FD0EDB2A04
:102E5000FE0E01E3DB2ADF2A010E01E3DB2A1E0E50
:102E6000E66EE66A5CEC21F0E552E552DECF14F046
:102E7000DDCF15F0153404E214500E08000E155481
:102E800001E201D0C9D7020EE15C02E2E16AE5523B
:102E9000E16EE552E7CFD9FF12008B908B948B92B5
:102EA0008B9A899A8B948B84210EE66EC5D8E55255
:102EB000B10EE66EC1D8E552040EE66EBDD8E552FD
:102EC000140EE66EB9D8E5520C0EE66EB5D8E55292
:102ED000200EE66EB1D8E5520C0EE66EADD8E55286
:102EE0001200D9CFE6FFE1CFD9FF020EE1268B8297
:102EF0008B908B94FA0EE66EE66A80EC21F0E55238
:102F0000E5528B808B84C80EE66EE66A80EC21F079
:102F1000E552E552210EE66E8FD8E552900EE66E30
:102F20008BD8E552040EE66E87D8E552130EE66E96
:102F300083D8E5520C0EE66E7FD8E552200EE66E81
:102F40007BD8E552960EE66EE66A80EC21F0E552FB
:102F5000E5520C0EE66E70D8E552320EE66EE66A69
:102F600080EC21F0E552E552020EE15C02E2E16AFA
:102F7000E552E16EE552E7CFD9FF1200D9CFE6FF67
:102F8000E1CFD9FF040EE126FE0EDBCFE6FFC7D866
:102F9000E552D950FC0FE96EFF0EDA20EA6EEE50D2
:102FA000ED1001E13FD00C0E146E156AFC0EDBCF64
:102FB00008F0FD0EDBCF09F014C00DF015C00EF0C7
:102FC00078EC1CF008C0DEFF09C0DDFF020EDB6AF2
:102FD000030EDB6A020EDBCF14F0030EDBCF15F01D
:102FE000DECF16F0DDCF17F015501718E8AE02D07F
:102FF000173404D01650145C1750155813E2FE0E07
:10300000DBCFE6FF020EDBCFE6FF73D8E552E552D9
:103010003C0EE66E28D8E552020EDB2A030E01E3D1
:10302000DB2AD8D7040EE15C02E2E16AE552E16EE8
:10303000E552E7CFD9FF1200D9CFE6FFE1CFD9FFA4
:103040008B928B90190EE66EE66A5CEC21F0E552ED
:10305000E552FE0EDBCFE6FF1DD8E5528B80E55230
:10306000E7CFD9FF1200D9CFE6FFE1CFD9FF8B829E
:103070008B90190EE66EE66A5CEC21F0E552E552A3
:10308000FE0EDBCFE6FF06D8E5528B80E552E7CF98
:10309000D9FF1200D9CFE6FFE1CFD9FFE652080EE3
:1030A000DF6EDFCF14F0000EE76E1418E8AE02D02A
:1030B000143403D0E750D880145416E2899A0A0ECB
:1030C000E66EE66A5CEC21F0E552E552FE0EDBBEF0
:1030D00002D08B9A01D08B8A898ADB50020DFE0EBA
:1030E000F3CFDBFFDF06DDD7E552E552E7CFD9FFAF
:1030F0001200D9CFE6FFE1CFD9FFFD0EDB50070B61
:103100004009E66E99DFE552FE0EDB507F0B800929
:10311000E66E92DFE552E552E7CFD9FF1200D9CF34
:10312000E6FFE1CFD9FFE652DF6ADFCF14F0540E9D
:10313000E76E1418E8AE02D0E73402D0E750145C12
:1031400020E2FE0EDBCFE6FFDFCFE6FFD2DFE55267
:10315000E5520A0EE66EE66A5CEC21F0E552E552B5
:10316000E66A200EE66EA9D8E552E5520A0EE66E32
:10317000E66A5CEC21F0E552E552060EDF24DF6ED4
:10318000D4D7FE0EDBCFE6FFE66AB3DFE552E552A9
:10319000E552E552E7CFD9FF1200D9CFE6FFE1CFE4
:1031A000D9FF020EE126E66AE66AA3DFE552E552A0
:1031B000DE6ADD6ADECF14F0DDCF15F0D890155051
:1031C00004E6050E145C000E15582FE2E66A4BDF8C
:1031D000E552E66A48DFE552E66A45DFE552E66A0F
:1031E00042DFE552E66A3FDFE552E66A3CDFE55240
:1031F000E66A39DFE552E66A36DFE552E66A33DF32
:10320000E552E66A30DFE552E66A2DDFE552E66A0E
:103210002ADFE552E66A27DFE552E66A24DFE55257
:10322000DF2A010E01E3DB2AC5D7E66AE66A61DF21
:10323000E552E552020EE15C02E2E16AE552E16E1E
:10324000E552E7CFD9FF1200D9CFE6FFE1CFD9FF92
:10325000E652DF6ADFCF14F0080EE76E1418E8AE0E
:1032600002D0E73402D0E750145C22E2DFCFE6FF61
:10327000FE0EDBCFE6FF3DDFE552E552E66AF3DE08
:10328000E552E66AF0DEE552E66AEDDEE552E66A10
:10329000EADEE552E66AE7DEE552E66AE4DEE5529A
:1032A000E66AE1DEE552E66ADEDEE552DF2AD2D7E3
:1032B000E552E552E7CFD9FF1200D9CFE6FFE1CFC3
:1032C000D9FFFE0EDB500C01C26FC36B200EC25D36
:1032D000000EC35901E24DD07F0ED880C255000EBA
:1032E000C35501E246D0C46BC56B050EC45D000E2C
:1032F000C5593CE2C2CCC6FCC3CCC7FC200EC65F9D
:10330000000EC75B050EC703F3CFC7FCC603F3CFA0
:10331000C6FCF450C727C651C425F66EC751C52157
:10332000F76E5D0EF6263E0EF7220800F5CFC8FCBC
:10333000C96BC8BFC969C8CCE6FF95DEE552FD0E72
:10334000DBCF14F0000EE76E1418E8AE02D0143490
:1033500003D0E750D880145404E2C8CCE6FF83DEE3
:10336000E5520C01C42B000EC523BFD7E66A7BDEF5
:10337000E552E552E7CFD9FF1200D9CFE6FFE1CF02
:10338000D9FFE6528B828B90080EDF6EDFCF14F0F0
:10339000000EE76E1418E8AE02D0143403D0E750E4
:1033A000D880145417E2899A0A0EE66EE66A5CEC3D
:1033B00021F0E552E552FE0EDBB002D08B9A01D02F
:1033C0008B8A898ADB407F0BE76EFE0EE7CFDBFF3F
:1033D000DF06DCD78B80E552E552E7CFD9FF12003C
:1033E000E66A9DDEE552010EE66E99DEE552020EBA
:1033F000E66E95DEE552030EE66E91DEE552040EB2
:10340000E66E8DDEE552050EE66E89DEE552060EAD
:10341000E66E85DEE552070EE66E81DEE5521200AD
:10342000D9CFE6FFE1CFD9FFFD0EDBCFE6FFFE0EE1
:10343000DBCFE6FF5EDEE552E552E66A200EE66E81
:103440003CDFE552E552FD0EDBCFE6FFFE0EDBCFA3
:10345000E6FF4FDEE552E552E552E7CFD9FF120015
:10346000E66A01DEE552040EE66EFDDDE552020E6F
:10347000E66EF9DDE5527F0EE66EF5DDE552020EF1
:10348000E66EF1DDE552040EE66EEDDDE552E66A2C
:10349000EADDE552E66AE7DDE5521200100EE66E5F
:1034A000E2DDE552200EE66EDEDDE5527F0EE66ED1
:1034B000DADDE552200EE66ED6DDE552100EE66E40
:1034C000D2DDE552E66ACFDDE552E66ACCDDE552B3
:1034D000E66AC9DDE5521200080EE66EC4DDE5526B
:1034E0001C0EE66EC0DDE5522A0EE66EBCDDE5522E
:1034F000080EE66EB8DDE552080EE66EB4DDE55264
:10350000F80EE66EB0DDE552E66AADDDE552E66A3C
:10351000AADDE5521200080EE66EA5DDE552080EA2
:10352000E66EA1DDE5522A0EE66E9DDDE5521C0E2B
:10353000E66E99DDE552080EE66E95DDE552E66A27
:1035400092DDE552E66A8FDDE552E66A8CDDE552F2
:103550001200E66A88DDE552060EE66E84DDE5526D
:10356000090EE66E80DDE552090EE66E7CDDE55261
:10357000060EE66E78DDE552E66A75DDE552E66A2E
:1035800072DDE552E66A6FDDE5521200E66A6BDD38
:10359000E552060EE66E67DDE5520F0EE66E63DD60
:1035A000E5520F0EE66E5FDDE552060EE66E5BDD60
:1035B000E552E66A58DDE552E66A55DDE552E66A0F
:1035C00052DDE5521200D9CFE6FFE1CFD9FFFD0E63
:1035D000DBCFE9FFFE0EDBCFEAFFEF5019E0FC0E78
:1035E000DBCFE6FFFD0EDBCFE9FFDB2AFE0EDBCFF4
:1035F000EAFF01E3DB2AEF50E66E5FDEE552E552BB
:103600000A0EE66EE66A5CEC21F0E552E552DFD781
:10361000E552E7CFD9FF1200019E08D0019E09AE06
:1036200005D0086C091EE86A0922018E09C003F062
:1036300008C002F0136A126A8E0E046E056A50EF1B
:103640001DF00F7E016A8CEC1DF0A4EC1DF001B69C
:1036500034EF1DF001A20AD001AA03D001BE34EF5D
:103660001DF001A440EF1DF03DEF1DF001AA05D0B3
:1036700001AC40EF1DF03DEF1DF001A00AD001A804
:1036800008D001BE04D001A402D049EF1DF04DEFD7
:103690001DF0126A056A0F500A5C116E10E307C034
:1036A00013F008C002F009C003F00AC010F00CC00B
:1036B00007F00DC008F00EC009F0013A09D00CC0A7
:1036C00013F00DC002F00EC003F00FC010F0116C2B
:1036D000019E01BC018E10C004F001B07CEF1DF012
:1036E0001A0E11607CEF1DF0046A0A6A01A408D06A
:1036F000076C081E091E0A1EE86A082209220A220F
:1037000001AC08D0136C021E031E041EE86A0222DC
:1037100003220422066A115207E00A3409320832F1
:1037200007320632112EF9D707501326085002220D
:10373000095003220A50042206C012F0019E04AE72
:103740000BD0126C131E021E031E041EE86A132205
:10375000022203220422018E04A006D0D880033264
:10376000023213321232102A10C004F050EF1DF052
:10377000016A8CEC1DF0A4EC1DF001B634EF1DF0D5
:1037800001A205D001BA34EF1DF03BEF1DF001BAE4
:1037900047EF1DF001A005D001B834EF1DF047EF51
:1037A0001DF001B83BEF1DF0056A7F0E0A24046E80
:1037B000E86A05220F50045EE86A055A1A0E106E78
:1037C0000A6A126A136A026A036A0C50075E0D5095
:1037D000085A0E50095A000E0A5A09E70C500726DB
:1037E0000D5008220E500922000E0A2201D0128A22
:1037F000D8900736083609360A36D890123613366E
:1038000002360336102EE1D7095008100710D8A44D
:10381000128A50EF1DF0016A8CEC1DF0A4EC1DF033
:1038200001B634EF1DF001A205D001B834EF1DF050
:103830003BEF1DF001AA05D001B034EF1DF03BEFC6
:103840001DF001B002D001A802D047EF1DF0056ABB
:103850000F500A24046EE86A05227E0E045EE86AB0
:10386000055A126A136A026A036A0E500902F4CFFB
:1038700003F0F3CF02F00D500902F3501326F45079
:103880000222000E03220E500802F3501326F450B9
:103890000222000E03220C500902F3501226F450AB
:1038A0001322000E022203220D500802F3501226AA
:1038B000F4501322000E022203220E500702F3508E
:1038C0001226F4501322000E022203220C5008028A
:1038D000F4501226000E1322022203220D5007027A
:1038E000F4501226000E13220222032250EF1DF084
:1038F000006A0EAE81EF1CF00D6C0E1EE86A0E22FF
:10390000001E09AE89EF1CF0086C091EE86A092246
:10391000001E81EC24F009BE99EF1CF000AE000CF3
:10392000086C091EE86A0922046C051EE86A052273
:10393000000C00BE90EF1CF00188FF0C016A8CECBB
:103940001DF001B6A8EF1CF001A20ED001B405D005
:103950007F0E096EFF0E086E1FD0800E096E086A7A
:103960001BD0096A086A18D001B0FBD78F0E0A6015
:10397000EDD77E0E0A64F5D78E0E0A5C05E0D8906E
:10398000093208320A2AF8D701A406D0086C091EA9
:10399000E86A092209AEE5D71200DFEC1CF001B697
:1039A000000C01B0000C01B4000C010CDFEC1CF0A9
:1039B00001B6000C01B0000C01A4000C010C016A5E
:1039C0008CEC1DF0A4EC1DF001B6120001AE08D085
:1039D00001A004D001A802D00180120001901200C1
:1039E0000F500A5C0BE10E50095C08E10D50085CB9
:1039F00005E10C50075C02E101801200D8A002D062
:103A0000018E10D00A500FC00AF00F6E09500EC080
:103A100009F00E6E08500DC008F00D6E07500CC076
:103A200007F00C6E0F500A5C10E0FF0F09E00190E8
:103A300001B403D001AE0184120001AE0194120062
:103A40000F2AD8900E320D320C320C50075E0D50FA
:103A5000085A0E50095A09BEEAD7D89007360836D8
:103A600009360A2EF8D7C8D77F0E0A6EFF0E096EE8
:103A7000086E076E12007F0E01BEFF0E0A6E02D0A6
:103A80007F0E0A6E800E096E086A076AF3D701AED0
:103A900004D0800E0A6E096AF7D70A6A096AF4D759
:103AA0000350021013101210F8E005BEF0D703BE49
:103AB0000CD004500510EBE0D890123613360236C5
:103AC00003360406D8A00506F2D70550D4E1042831
:103AD000D2E012AE11D07F0E121402E113A00CD06E
:103AE000132AE86A0222032207E3D8800332023253
:103AF0001332042A0428BFE00450C9E013C007F0C1
:103B000002C008F00334096E04300A6E09320A9EBE
:103B100001BE0A8E3AEF1DF009360A3602E301842F
:103B2000017E06E101800A6A096A086A076A1200D2
:103B30000A2803E0D88009321200D890093202E145
:103B400001821200018612000E360F3602E3018C4C
:103B5000017E06E101880F6A0E6A0D6A0C6A120086
:103B60000F2803E0D8800E321200D8900E32EAE11E
:103B7000018A120009C013F008C012F008500D02AB
:103B8000F4CF07F0F3CF06F009500E02F4CF09F09E
:103B9000F3CF08F00D02F3500726F4500822E86A2C
:103BA000092212500E02F3500726F4500822E86A48
:103BB00009220EAEE0EF1DF01250085E1350095AB4
:103BC00013AE000C0D50085E0E50095A000C4C69E3
:103BD0006E6B20524E343120424144004C696E6B72
:103BE00020524E3431204F4B00474B0041747465D6
:103BF0006E746520646174612066726F6D20524E30
:103C000034310D0A004D657375726573204C6F6316
:103C1000616C6573203A20454130203D20252035D8
:103C20006420204541313D252035640D0A00496E50
:103C3000697420414443302065742041444331205D
:103C40004D65737572652064652074656D6572617C
:103C500074757265730D0A00496E6974204144439E
:103C600030204144433100496E69742042542D484C
:103C70004330352D426C6575207465726D696EE94F
:103C80006520424144202C207265746F75723D2579
:103C90002031640D0A00496E697420484330354272
:103CA0002042414400496E69742042542D484330FB
:103CB000352D426C6575207465726D696EE96520FD
:103CC0004F4B202C207265746F75723D2520316436
:103CD0000D0A00496E6974204843303542204F4B2D
:103CE0002000496E69742061766563207465737481
:103CF00020666565646261636B20647520204254B0
:103D00002D48433035206D6F646520536C617665B6
:103D10000D0A00554152543220656E20657370695A
:103D20006F6E200D0A00403D393844333331423143
:103D30003744363900494E49542E484330352042E5
:103D40004C455500494E49542E554152543220207D
:103D50002020005665722E31343034313320433107
:103D60003800524E34312D48433035204C494E4BAB
:103D7000004E4F4B4941353131302031384620001B
:103D80002E2E2E2E2E2E3F2E2E2E2E2E2E2E00207E
:103D900020202020202020202020202020004574CA
:103DA000617065203409004F4B6C696E766F7256F6
:103DB0000041542B56455253494F4E004574617093
:103DC00065203309004F4B7365746E616D6500416A
:103DD000542B4E414D45484330352D374436392D0F
:103DE00042004574617065203209004F4B73657461
:103DF00050494E0041542B50494E35363738004516
:103E000074617065203109004F4B004154004574C6
:103E10006170653A2030207375722034000D0A00FD
:103E20004E625F576174743B54656D705F65787462
:103E30003B4E625F43686175666665730D0A004CB0
:103E400065637475726520456570726F6D205049A9
:103E500043202049783D253035640D0A00000000DC
:103E6000000000005F00000007000700147F147FBF
:103E700014242A7F2A1223130864623649552250DB
:103E80000005030000001C2241000041221C001418
:103E9000083E081408083E080800503000000808D2
:103EA000080808006060000020100804023E514924
:103EB000453E00427F400042615149462141454B09
:103EC000311814127F1027454545393C4A4949307D
:103ED00001710905033649494936064949291E0039
:103EE0003636000000563600000814224100141433
:103EF00014141400412214080201510906324979B0
:103F0000413E7E1111117E7F494949363E41414172
:103F1000227F4141221C7F494949417F090909010A
:103F20003E4149497A7F0808087F00417F410020CF
:103F300040413F017F081422417F404040407F02C2
:103F40000C027F7F0408107F3E4141413E7F0909FA
:103F500009063E4151215E7F0919294646494949D2
:103F60003101017F01013F4040403F1F2040201FA1
:103F70003F4038403F631408146307087008076126
:103F800051494543007F414100020408102000418F
:103F9000417F000402010204404040404000010211
:103FA000040020545454787F4844443838444444EE
:103FB00020384444487F3854545418087E0901027C
:103FC0000C5252523E7F0804047800447D40002089
:103FD00040443D007F1028440000417F40007C04A5
:103FE0001804787C0804047838444444387C141459
:103FF0001408081414187C7C080404084854545409
:1040000020043F4440203C4040207C1C2040201C99
:104010003C4030403C44281028440C5050503C4414
:1040200064544C44000836410000007F0000004109
:1040300036080010080810087846414678464F5365
:104040004320696E7465726E652031364D487A0D75
:1040500000506F727420486172642055415254318F
:104060002031393230302C4E2C382C31202852431C
:104070003620524337202D3E20425420524E3431B8
:10408000200D0A00506F72742048617264205541FF
:1040900052543220200D0A00496E69742041444375
:1040A0003020657420414443310D0A0020313846E8
:1040B00032364B32325F4E6F6B6961353131305F72
:1040C00042545F484330355F374436395F425F3191
:1040D00034303431325F31364D687A2E630D0A0048
:1040E00041726D656D656E7420495420554152547E
:1040F00032200D0A2000202031384632364B323231
:104100005F4E6F6B6961353131305F42545F4843B8
:1041100030355F374436395F425F313430343132C5
:104120005F31364D687A2E630D0A00200020002092
:1041300031384632364B32325F484330355F536C4C
:104140006176655F323031342E6D63700D0A000088
:104150005665722E313430343133204331382020CB
:1041600020202020202020202020200D0A00004A8E
:10417000616E762E00466576722E004D6172732058
:1041800000417672696C004D61692020004A7569B2
:104190006E20004A75696C2E00416F7574200053C3
:1041A0006570742E004F63746F2E004E6F76652E0F
:1041B00000446563652E0044696D616E004C756E48
:1041C0006469004D61726469004D65726372004AF2
:1041D000657564690056656E64720053616D65644F
:1041E00000FFFB0EE3CFF6FFFC0EE3CFF7FFFD0E63
:1041F000E3CFF8FFFE0EE3CFE9FFFF0EE3CFEAFFC8
:10420000F90EE35003E1FA0EE35009E0F90EE3067C
:1042100002E2FA0EE3060900F550EE5CF1E012004E
:10422000FB0EE3CFF6FFFC0EE3CFF7FFFD0EE3CF6F
:10423000F8FFFE0EE3CFE9FFFF0EE3CFEAFFE9CF81
:10424000F3FFEACFF4FF0900F5CFEFFFEE66FBD7EF
:104250001200FE0EE3CFE9FFFF0EE3CFEAFFF36AA1
:10426000F46AEE5203E0F34AF42AFBD71200FF0E81
:10427000E3CFF8FFE552FF0EE3CFF7FFE552FF0E65
:10428000E3CFF6FFE552E66AE66AE66A0900F55210
:1042900009E0FD0EE32A05E1FE0EE32A02E1FF0E2E
:1042A000E32AF4D7FD0EE3CF07F0FE0EE3CF08F0CC
:1042B000FF0EE3CF09F01200D9CFE6FFE1CFD9FF1F
:1042C000020EE126FD0EDBCFDEFFDBCFDDFFD9CF17
:1042D000E9FFDACFEAFFEE06000EED5AEECF14F05A
:1042E000EDCF15F01450151001E0F1D7020EE15C8E
:1042F00002E2E16AE552E16EE552E7CFD9FF120032
:10430000D9CFE6FFE1CFD9FFF29A010ED56EFC0EB0
:10431000D76E190ED66ED950FD0FE96EFF0EDA205A
:10432000EA6E000ED880EE54000EED540EE2D58EEB
:10433000F2A4FED7F294FD0EDB06FE0E01E2DB06D0
:10434000FC0ED76E190ED66EE6D7D56AE552E7CFCA
:10435000D9FF1200F29A070ED56EC20ED76EF70E75
:10436000D66ED58EF2A4FED7F294D56AC20ED76E61
:10437000F70ED66E1200D9CFE6FFDACFE6FFE1CF17
:10438000D9FFE2CFDAFFE652E652E652E652D950C2
:10439000F90F146EFF0EDA20156E020E14C0DBFF4B
:1043A000030E15C0DBFF020EDBCFE6FF030EDBCFF3
:1043B000E6FFF90EDBCFE6FFFA0EDBCFE6FFFB0EE2
:1043C000DBCFE6FFD950FC0FE66EFF0EDA20E66E7B
:1043D000BBEC10F0146E070EE15C02E2E16AE552FC
:1043E000E16E1450F3CFDEFFF4CFDDFFFC0EDBCF28
:1043F000E9FFFD0EDBCFEAFFEF6ADECF14F0DDCF81
:1044000015F014C0F3FF15C0F4FF040EE15C02E2E6
:10441000E16AE552E16EE552E5CFDAFFE7CFD9FF79
:1044200012000E0EF66E000EF76E000EF86E0F0103
:104430000900F550056F0900F550066F03E10567A7
:1044400001D03DD00900F550006F0900F550016F13
:104450000900F550026F09000900F550E96E0900E6
:10446000F550EA6E090009000900F550036F0900D4
:10447000F550046F09000900F6CF07FFF7CF08FFDA
:10448000F8CF09FF00CFF6FF01CFF7FF02CFF8FF0B
:104490000F01035302E1045307E00900F550EE6EEB
:1044A0000307F8E20407F9D707CFF6FF08CFF7FFB5
:1044B00009CFF8FF0F010507000E065BBFD71200FA
:1044C000D9CFE6FFDACFE6FFE1CFD9FFE2CFDAFFBF
:1044D000E652E652E652E652D950F90F146EFF0E3C
:1044E000DA20156E14C0DEFFDD6EDECFE6FFDDCF15
:1044F000E6FFF90EDBCFE6FFFA0EDBCFE6FFFB0EA1
:10450000DBCFE6FFFC0EDBCFE6FFFD0EDBCFE6FFE9
:10451000BBEC10F0146E070EE15C02E2E16AE552BA
:10452000E16E1450020EF3CFDBFF030EF4CFDBFF7E
:10453000020EDBCF14F0030EDBCF15F014C0F3FF37
:1045400015C0F4FF040EE15C02E2E16AE552E16E9F
:10455000E552E5CFDAFFE7CFD9FF1200D9CFE6FF6A
:10456000DACFE6FFE1CFD9FFE2CFDAFFFB0EDBCFF8
:1045700014F0FC0EDBCF15F00001800E15141AE1CB
:10458000FB0EDBCFE9FFFC0EDBCFEAFFEECFF3FF44
:10459000EDCFF4FFEE2A000EEF22F3CFE9FFF4CFC8
:1045A000EAFFFD0EDBCFEFFFEF50156AF36E15C08B
:1045B000F4FF10D0FB0EDB50FE0806E1FD0EDBCF52
:1045C000E6FFD7EC24F005D0FD0EDBCFE6FF03ECD1
:1045D00000F0E552E552E5CFDAFFE7CFD9FF120050
:1045E000D9CFE6FFDACFE6FFE1CFD9FFE2CFDAFF9E
:1045F000726A716AFD0EDBB07288DBA202D0728C27
:10460000718CDBB4728EDBA602D0718801D0718A06
:10461000DBA802D0728401D07294DBBA7186DBAC65
:1046200002D0A38A01D0A39ADBAE02D0A38801D026
:10463000A398FB0EDB50756EFC0EDBCF15F015C09A
:1046400014F0156A1450766E728A718EE552E5CFB9
:10465000DAFFE7CFD9FF1200D9CFE6FFDACFE6FFC6
:10466000E1CFD9FFE2CFDAFFAC6AAB6AFD0EDBB077
:10467000AC88DBA202D0AC8CAB8CDBB4AC8EDBA6FE
:1046800002D0AB8801D0AB8ADBB8AC84DBBAAB8696
:10469000DBAC02D09D8A01D09D9ADBAE02D09D8812
:1046A00001D09D98FB0EDB50AF6EFC0EDBCF15F0FA
:1046B00015C014F0156A1450B06EAC8AAB8EE5527A
:1046C000E5CFDAFFE7CFD9FF120006500B02F3CF98
:1046D00002F0F4CF03F00C02F3500326000EF42096
:1046E000046E06500D02F3500426000EF420056EF1
:1046F00006500E02F350052607500B02F350032616
:10470000F4500422000E052207500C02F350042638
:10471000F450052207500D02F350052608500B02F5
:10472000F3500426F450052208500C02F3500526DD
:1047300009500B02F35005261200056A046A036A49
:10474000026A200EE76ED89006360736083609361C
:1047500002360336043605360B50025C0C50035803
:104760000D5004580E50055809E30B50025E0C50D2
:10477000035A0D50045A0E50055A062AE72EE4D764
:104780001200D9CFE6FFDACFE6FFE1CFD9FFE2CFC3
:10479000DAFFE652F20E0C01F91771AC03D0F99171
:1047A00071B0F98171B4F98571B2F9877450DF6E17
:1047B000DF50E552E552E5CFDAFFE7CFD9FF12002F
:1047C000D9CFE6FFDACFE6FFE1CFD9FFE2CFDAFFBC
:1047D000E652F20E0C01FA17ABAC03D0FA91ABB073
:1047E000FA81ABB4FA85ABB2FA87AE50DF6EDF5018
:1047F000E552E552E5CFDAFFE7CFD9FF1200D9CF76
:10480000E6FFDACFE6FFE1CFD9FFE2CFDAFFE652EB
:10481000E652FC0EDBCFDEFFDBCFDDFF010EDB500F
:10482000B36EDF50B26EE552E552E552E5CFDAFFE6
:10483000E7CFD9FF1200D9CFE6FFDACFE6FFE1CF0D
:10484000D9FFE2CFDAFFE652E652FC0EDBCFDEFF05
:10485000DBCFDDFF010EDB50CF6EDF50CE6EE552B9
:10486000E552E552E5CFDAFFE7CFD9FF1200D9CF05
:10487000E6FFDACFE6FFE1CFD9FFE2CFDAFFE6527B
:10488000E652FC0EDBCFDEFFDBCFDDFF010EDB509F
:10489000D76EDF50D66EE552E552E552E5CFDAFF2E
:1048A000E7CFD9FF1200D9CFE6FFDACFE6FFE1CF9D
:1048B000D9FFE2CFDAFF72AC04D072900C01F9B3E9
:1048C0007280FD0EDB50736EE552E5CFDAFFE7CF65
:1048D000D9FF1200D9CFE6FFDACFE6FFE1CFD9FF4B
:1048E000E2CFDAFFACAC04D0AC900C01FAB3AC80F0
:1048F000FD0EDB50AD6EE552E5CFDAFFE7CFD9FF15
:104900001200056A046A100EE76ED8900836093660
:10491000043605360D50045C0E50055805E30D5065
:10492000045E0E50055A082AE72EF0D71200F36AEB
:10493000F46AFF0EE124E96EFF0EE220EA6EED66F6
:1049400007D02F0EEF6404D03A0EEF6001D0F32AA7
:104950001200FF0EE3501C6E480E01D04C0EE76EA5
:10496000E72EFED7E76AE72EFED71C2EF7D700000A
:104970001200380EF36E00EE00F00F0E01D8120098
:10498000EA6002D0EE6AFCD7F350E9601200EE6AEA
:10499000FCD71EEE00F02EEE00F0F86A019C11EC40
:1049A00022F009EC25F0BFEC0BF0FBD71200FF0E54
:1049B000E350ACBA04D0AF6AAB8EAC8A949CACA284
:1049C000FED7AD6EF36EF46A1200FF0EE350E84EB0
:1049D0001200000000D000D000D0E82EFAD712005C
:1049E000C450176E166AC3501610F36E17C0F4FF4A
:1049F000120030313233343536373839616263640E
:104A0000656600FFC250020B01E0010E1200C28277
:104A100012001200000000000000005F000000070C
:104A2000000700147F147F14242A7F2A12231308FE
:104A3000646236495522500005030000001C2241E3
:104A4000000041221C0014083E081408083E080813
:104A500000503000000808080808006060000020CE
:104A6000100804023E5149453E00427F4000426129
:104A70005149462141454B311814127F10274545B5
:104A800045393C4A494930017109050336494949CC
:104A900036064949291E0036360000005636000009
:104AA00008142241001414141414004122140802A2
:104AB00001510906324979413E7E1111117E7F492B
:104AC0004949363E414141227F4141221C7F4949AB
:104AD00049417F090909013E4149497A7F0808088F
:104AE0007F00417F41002040413F017F0814224167
:104AF0007F404040407F020C027F7F0408107F3ED1
:104B00004141413E7F090909063E4151215E7F092D
:104B1000192946464949493101017F01013F404079
:104B2000403F1F2040201F3F4038403F631408147F
:104B30006307087008076151494543007F41410000
:104B400002040810200041417F00040201020440D9
:104B500040404040000102040020545454787F48F3
:104B60004444383844444420384444487F385454FA
:104B70005418087E0901020C5252523E7F08040468
:104B80007800447D40002040443D007F10284400D0
:104B900000417F40007C041804787C0804047838C5
:104BA000444444387C14141408081414187C7C08F9
:104BB0000404084854545420043F4440203C4040DE
:104BC000207C1C2040201C3C4030403C44281028C5
:104BD000440C5050503C4464544C4400083641004E
:104BE00000007F0000004136080010080810087817
:104BF00046414678000000003D40514084409840C6
:104C0000AC40E040F6402B412D412F415041000087
:104C1000FFFFFFFFFFFFFFFFFFFFFFFFFFFFFFFFA4
:104C2000FFFFFFFFFFFFFFFFFFFFFFFFFFFFFFFF94
:104C3000FFFFFFFFFFFFFFFFFFFFFFFFFFFFFFFF84
:104C4000FFFFFFFFFFFFFFFFFFFFFFFFFFFFFFFF74
:0200000400F00A
:100000000000FFFFFFFFFFFFFFFFFFFFFFFFFFFFFE
:10001000FFFFFFFFFFFFFFFFFFFFFFFFFFFFFFFFF0
:10002000FFFFFFFFFFFFFFFFFFFFFFFFFFFFFFFFE0
:10003000FFFFFFFFFFFFFFFFFFFFFFFFFFFFFFFFD0
:10004000FFFFFFFFFFFFFFFFFFFFFFFFFFFFFFFFC0
:1003E0007061756C666A756A6F40667265652E66C7
:1003F000722020202020202020202020200D00FFFF
:020000040030CA
:0E0000000028193C009D84000FC00FE00F4047
:020000040020DA
:08000000FFFFFFFFFFFFFFFF00
:00000001FF
